:020000040800F2
:100000007006002091010008710B00086D0B0008BC
:100010006F0B0008C9080008111400080000000058
:10002000000000000000000000000000710E000849
:1000300061090008000000001D0C0008750E000892
:10004000AB010008AB010008AB010008AB010008E0
:10005000AB010008AB01000865090008AB0100080E
:10006000AB010008AB010008AB010008AB010008C0
:10007000AB010008AB010008AB010008AB010008B0
:10008000AB010008AB010008AB010008AB010008A0
:10009000AB010008AB010008AB010008AB01000890
:1000A000AB010008AB010008AB010008AB01000880
:1000B000AB010008AB0100085D0F0008AB010008B0
:1000C000AB010008AB010008AB010008AB01000860
:1000D000AB010008AB010008AB010008AB01000850
:1000E000AB010008AB010008AB01000800F002F80A
:1000F00000F03EF80AA090E8000C82448344AAF184
:100100000107DA4501D100F033F8AFF2090EBAE881
:100110000F0013F0010F18BFFB1A43F0010318473B
:100120006C1A00008C1A0000103A24BF78C878C1FD
:10013000FAD8520724BF30C830C144BF04680C60ED
:10014000704700000023002400250026103A28BF35
:1001500078C1FBD8520728BF30C148BF0B60704739
:100160001FB59DE8030000F0BDF91FBD10B510BD1F
:1001700000F076F91146FFF7F3FF01F088FC00F07C
:10018000E7F903B4FFF7F2FF03BC01F07DFC0000C8
:100190000948804709480047FEE7FEE7FEE7FEE71B
:1001A000FEE7FEE7FEE7FEE7FEE7FEE70448054957
:1001B000054A064B704700008D0E0008ED00000850
:1001C00070000020700600207002002070020020E5
:1001D000704710B54C1084EA530404D54042C1F175
:1001E000000138BF491E1B4204D55242C3F100032F
:1001F00038BF5B1E00F036F814F0804F04D0404248
:10020000C1F1000138BF491E14F0004F04D0524222
:10021000C3F1000338BF5B1E10BD4FF0000204297C
:10022000C0F0128010F0030C00F09580CCF1040CAB
:10023000BCF1020F18BF00F8012BA8BF20F8022B59
:10024000A1EB0C0100F087B85FEAC17C24BF00F885
:10025000012B00F8012B48BF00F8012B70477047B5
:100260007047704753EA020C00F069802DE9F04BAB
:100270004FF00006002B1FBFB3FA83F503FA05F415
:1002800024FA05F65E4012BF1643B2FA82F502FA6E
:1002900005F4C5F120051EBF22FA05FC44EA0C0452
:1002A000203556EA044C4FEA144418BF641C4FF042
:1002B00000084FF00009904271EB030C39D300297C
:1002C00019BFB1FA81F701FA07F6B0FA80F700FA20
:1002D00007F6C7F120071EBF20FA07FC46EA0C0606
:1002E0002037B6FBF4FCA7EB0507103F07F01F0B08
:1002F000CBF120060CFA0BFB2CFA06F644BFB346F2
:100300000026202FA4BF5E464FF0000B5BEA060CD0
:1003100008BF4FF0010B19EB0B09ABFB027C48EB5C
:100320000608C01B06FB02CC0BFB03CC71EB0C01D7
:10033000C1E70B46024641464846BDE8F08B13B57F
:100340004FF000004FF00001AFF30080BDE81C400B
:1003500070474FF0000200B5134694469646203988
:1003600022BFA0E80C50A0E80C50B1F12001BFF46E
:10037000F7AF090728BFA0E80C5048BF0CC05DF8D4
:1003800004EB890028BF40F8042B08BF704748BF22
:1003900020F8022B11F0804F18BF00F8012B704796
:1003A000004870474400002070B5064600F07EF813
:1003B000056806F10B0020F00704B4429CBF002042
:1003C00070BD2B466A68BAB11068A04210D304F120
:1003D000080188423CBF5068586007D35168101923
:1003E00041601168091B016058601460101D70BDE8
:1003F00013465268002AE7D12146284600F05EF8ED
:100400000028DED170BD70B50446051F00F04EF81F
:100410000068002C14BF446870BD002C18BFAC42AB
:100420003CBF20466468F8D301680A18AA4218BF86
:10043000456003D12A6805461144016028684119C6
:10044000A1421CBF6C6070BD61686960216808448E
:10045000286070BD00F082B800487047100000208E
:100460007546FFF7F9FFAE4605006946534620F092
:100470000700854618B020B5FFF798FEBDE820407C
:100480004FF000064FF000074FF000084FF0000B50
:1004900021F00701AC46ACE8C009ACE8C009ACE803
:1004A000C009ACE8C0098D4670470000004870479D
:1004B00018000020704770477047704738B50446F1
:1004C0000A4600206946AFF30080002808BF38BD07
:1004D00002460099204600F04EF8012038BD012068
:1004E00000F06BB8F8B5AFF30080054600200C466D
:1004F000102000BF0646A819A0420DD93246694611
:100500000020AFF30080070008BF00F056F8009805
:10051000A04218BF0546C419FFF7C8FF056007468B
:10052000F01D20F007004619284600F00AF8B442F2
:1005300008BFF8BDA21B31463868BDE8F84000F09E
:100540001AB800210160C0E90110704710207047FF
:100550000446AFF300802046FFF713FE10B500F00D
:1005600036F8016919B100220261884701E080680C
:10057000804700F01AF8034640688C46002818BFF0
:1005800088423CBF03464068F8D318681844884244
:1005900007D00CF1030020F00700001D411A521A89
:1005A0000146081D0A60FFF72EBF002000F03DF84D
:1005B000FFF7DCFD012001F067FA10B500F03CF810
:1005C000BDE8104000F02CB810B5FFF7EEFF70B595
:1005D00000F022F804680546A4B92020FFF7E4FEE5
:1005E000040011D0094900202C60C4E90001084929
:1005F000A1602073206160610649A06109B100F02B
:1006000043F8E061204670BDFFF7CFFF0000000017
:10061000C905000800000000004870474C00002099
:10062000002801D001F030BA704710B500F064F82E
:10063000BDE81040FFF7F4BF10B5012805D0002138
:1006400003A000F03FF8012010BD09A1F8E7000069
:1006500053494752544D454D3A204F7574206F66AB
:100660002068656170206D656D6F72790000000013
:100670003A2048656170206D656D6F727920636FF7
:10068000727275707465640010B58820FFF78CFE77
:10069000002801D00021017010BD802902D808B1C6
:1006A000017809B100207047012100F8081B70474C
:1006B00018B100F10802914201D0002070470021DA
:1006C0000170704770B505460C460A2000E06D1CAD
:1006D00001F0DBF935B128780028F8D102E0641C7C
:1006E00001F0D3F914B120780028F8D1BDE87040AA
:1006F0000A2001F0CAB9000010B5002102A0FFF7DE
:10070000E1FF012010BD0000534947414252543AD5
:100710002041626E6F726D616C207465726D696EDE
:100720006174696F6E0000000029816814BF41F098
:10073000010121F001018160704710B5A0F18041F5
:10074000B1F5923111D0B1F5806119D0B1F5A05158
:1007500018BF10BD0121C80300F090FABDE8104099
:1007600000214FF4004000F089BA0121480200F056
:1007700085FABDE8104000214FF4007000F07EBA09
:100780000121880200F07AFABDE8104000214FF400
:10079000806000F073BA0029816814BF41F48011B1
:1007A00021F480118160704701460020896811F0B2
:1007B000040F18BF01207047C06C80B2704702461A
:1007C000002012680A4218BF01207047014600202D
:1007D000896811F0080F18BF012070474268D1E9FD
:1007E000003C22F4807222F4702242EA0C221A4366
:1007F000426082680A4B1A40D1E903C343EA0C0302
:10080000D1F808C042EA4C021A438260C26A097DEC
:1008100022F47002491EC9B242EA0151C162704716
:10082000FDF7F1FF30B4072509290CD9C468A1F1FF
:100830000A0C0CEB4C0C05FA0CF5AC4303FA0CF368
:100840002343C36009E0046901EB410C05FA0CF590
:10085000AC4303FA0CF3234303614FF01F0C072A48
:100860000CD2436B521E02EB82020CFA02FC23EA0A
:100870000C0391401943416330BC70470D2A0CD2E0
:10088000036BD21F02EB82020CFA02FC23EA0C0378
:1008900091401943016330BC7047C36A0D3A02EBC3
:1008A00082020CFA02FC23EA0C0391401943C16254
:1008B00030BC7047816841F00801816070478168F1
:1008C00041F0040181607047FEE70000054A012302
:1008D00003FA00F00029116814BF084321EA000060
:1008E000106070470074004010B50121480700F007
:1008F000ADF9BDE8104000214FF0005000F0A6B95E
:100900000B4B10B41A6840F6FE7C0CFA00FC22EA8D
:100910000C02D1E900C44CEA040CD1E902412143A4
:100920004CEA010101FA00F01043186010BC704756
:1009300000740040A0F6F83081B000F1804000F56E
:1009400000400090016001B07047A0F6EC3081B02B
:1009500000F1804000F500400090016001B0704758
:100960007047000002490120087000F003B8000041
:100970000000002001490860704700001404014095
:10098000C368214A0168002B34D0136823EA0101AF
:100990001160111D0A6803689A430A60416801F1F9
:1009A000804101F582310A6803681A430A60174AD8
:1009B0001168036899431160131D1968D0F800C0CD
:1009C00021EA0C0119608168102908D001F18041E9
:1009D00001F582310A6800681043086070471168A9
:1009E000D0F800C041EA0C011160196800680843A2
:1009F00018607047406800F1804000F5823002685E
:100A000022EA01010160704700040140080401402E
:100A10008A0721F0030101F1804101F58031120FB5
:100A20000F23D1F808C093402CEA03038B608B6836
:100A300090401843886070472DE9F00191F808C094
:100A400000220CF00F031CF0100F1CBFD1F804C0E3
:100A50004CEA030391F800C04FF00F071CF0FF0FA2
:100A60004FF0010618BF04681CD00D8806FA02FC7E
:100A700005EA0C05654511D1950007FA05F824EA49
:100A8000080403FA05F52C438D68282D08BFC0F82B
:100A900014C003D0482D08BFC0F810C0521C082A4B
:100AA000E3D304600A88FF2A87BF44680022BDE8B8
:100AB000F001704702F1080C0D8806FA0CFC05EAFB
:100AC0000C05654511D1950007FA05F824EA0804DC
:100AD00003FA05F52C438D68282D08BFC0F814C013
:100AE0008D68482D08BFC0F810C0521C082AE1D3F9
:100AF0004460BDE8F001704770B4DFF86CC010F0DE
:100B0000004F14BFDCF81C20DCF80420C0F30344C1
:100B10004FF4401333EA00054FEA50534FEA0313F2
:100B200086B206FA03F316D010F4801F08BF9A436A
:100B300003D0032505FA04F4A24342F070620029B1
:100B400018BF1A4310F0004F14BFCCF81C20CCF88B
:100B5000042070BC7047DCF8044022F0706224F07E
:100B60007064CCF80440EAE700000140FEE7FEE7CD
:100B7000FEE7000010B4017842684FF00F0C01242A
:100B80002AB3194A126801F1E02102F4E062C2F5C9
:100B9000E062120AC2F104032CFA02F290F801C0DA
:100BA0000CFA03F390F802C00CEA02021A43120195
:100BB00081F80024007800F01F0104FA01F14009D7
:100BC000800000F1E020C0F8001110BC704701F077
:100BD0001F0004FA00F04909890001F1E021C1F881
:100BE000800110BC704700000CED00E0094B1A6852
:100BF00022F00302104318600748026842F0040222
:100C0000026001290CBF30BF20BF016821F0040140
:100C1000016070470070004010ED00E07047000078
:100C2000034A516821F44041084350607047000076
:100C300000100240044A0029D16914BF084321EA88
:100C40000000D0617047000000100240044A0029F3
:100C5000116914BF084321EA0000106170470000C9
:100C600000100240044A0029916914BF084321EA98
:100C7000000090617047000000100240044A002903
:100C8000D16814BF084321EA0000D060704700001B
:100C90000010024000224109094B012908BF1968D0
:100CA00003D002290CBF196A596A00F01F00012302
:100CB00003FA00F0084218BF0122104670470000F6
:100CC000001002400248406800F00C00704700002D
:100CD000001002400C490A6822F480320A600A6857
:100CE00022F480220A60B0F5803F04BF086840F417
:100CF000803006D0B0F5802F06BF086840F4A020F1
:100D00007047086070470000001002400149086603
:100D10007047000000004242034A516821F003017D
:100D200008435060704700000010024008B50020E2
:100D30000B4A00900020116811F4003F18BF0120F9
:100D40000099491C0091B1F5A06F01D00028F1D0A5
:100D50003120FFF79FFF002818BF012008BD0000C9
:100D60000010024010B504460B4884B0012150F831
:100D70002400FFF777FF0948694630F81400ADF802
:100D800000001020029003200190054850F8240034
:100D9000FFF752FE04B010BD441B00083A1B0008C8
:100DA000080000200349044A31F8101052F82000CE
:100DB000416170473A1B0008080000200349044ABB
:100DC00031F8101052F82000016170473A1B0008FA
:100DD0000800002030B504461F480D4689B050F881
:100DE0002400012140F00100FFF73CFF042008909F
:100DF0001A4806A930F81400ADF81800184850F841
:100E00002400FFF719FE012D1CBF09B030BD1548A5
:100E100010F81410801C10F81400FFF7F9FD1248A8
:100E2000012530F814000090002001900820CDE941
:100E300002056846FFF7A4FD0C4810F814008DF871
:100E400010000F208DF811008DF8120004A80595F0
:100E5000FFF790FE09B030BD401B0008341B0008AE
:100E600004000020301B0008361B0008381B000857
:100E7000704700000448807800284FF0000001D03F
:100E8000FFF79CBFFFF78EBF00000020304882B004
:100E9000016841F00101016042682E491140416042
:100EA000016821F4102121F080710160016821F4B2
:100EB00080210160416821F4FE0141604FF41F016F
:100EC00081600022C26200920192016841F4803187
:100ED0000160016801F4003101910099491C009101
:100EE000019919B90099B1F5A06FF2D1016811F417
:100EF000003F08BF019224D0012101914168416067
:100F00004168416041684160416821F47C11416061
:100F1000416841F498114160016841F080710160BD
:100F2000016811F0007FFBD0416821F003014160AE
:100F3000416841F002014160416801F00C0108295B
:100F4000FAD105494FF00060086002B07047000018
:100F5000001002400000FFF808ED00E010B50A4C58
:100F60000221204600F01AF9002808BF10BD022116
:100F7000204600F016F8054A012120465170BDE8D0
:100F80001040002100F010B80008004000000020D0
:100F90000029018814BF41F0800121F08001018007
:100FA0007047C943018270470029018814BF41F08E
:100FB000010121F001010180704710B5A0F18041CD
:100FC000B1F596313BD0B0F1804F4DD011F5943151
:100FD00040D0B1F5806151D0B1F5806158D0B1F504
:100FE00080615FD0B1F5806166D0B1F590316DD090
:100FF000B1F5C05175D0B1F580617DD0B1F580619A
:101000007DD011F59E317BD0B1F5806179D0B1F5FD
:10101000806177D0B1F5903175D0B1F5806173D032
:10102000B1F5806118BF10BD01218804FFF726FECD
:10103000BDE8104000214FF48020FFF71FBE0121C2
:10104000C802FFF71BFEBDE8104000214FF400600E
:10105000FFF714BE01210220FFF7F8FD0021BDE8D3
:1010600010400220FFF7F2BD01210846FFF7EEFD18
:101070000021BDE810400120FFF7E8BD0121042058
:10108000FFF7E4FD0021BDE810400420FFF7DEBDBE
:1010900001210820FFF7DAFD0021BDE810400820FB
:1010A000FFF7D4BD01211020FFF7D0FD0021BDE8DE
:1010B00010401020FFF7CABD01212020FFF7C6FD18
:1010C0000021BDE810402020FFF7C0BD01214803EA
:1010D000FFF7D4FDBDE8104000214FF40050FFF7AA
:1010E000CDBD0121C804FFF7C9FDBDE810400021B6
:1010F0004FF40020FFF7C2BD0121080505E00DE017
:1011000017E020E029E033E03DE0FFF7B7FDBDE860
:10111000104000214FF48010FFF7B0BD01214805B9
:10112000FFF7ACFDBDE8104000214FF40010FFF7C1
:10113000A5BD01214020FFF789FD0021BDE8104039
:101140004020FFF783BD01218020FFF77FFD0021B4
:10115000BDE810408020FFF779BD01210802FFF7AC
:1011600075FDBDE8104000214FF48070FFF76EBDA3
:1011700001210804FFF782FDBDE8104000214FF473
:101180008030FFF77BBD01214804FFF777FDBDE804
:10119000104000214FF40030FFF770BD038A002299
:1011A00080890B4200EA01001CBF00280122104682
:1011B0007047002A828914BF114322EA010181810C
:1011C000704710B4028C22F001020284028C8388E2
:1011D000B0F818C00C882CF0730C44EA0C0C0C8985
:1011E00022F0020222434C882243A0F18044B4F54D
:1011F00096341CBFA0F18044B4F59A340DD0A0F110
:101200008044B4F5A0341FBFA0F18044B4F5A234EB
:10121000A0F18044B4F5A4340DD14C8922F0080229
:1012200022438C8822F0040222438C8923F44073E9
:101230002343CC8923438380A0F818C0C9888186C2
:10124000028410BC704730B4028C22F01002028479
:10125000028C8388B0F818C00D882CF4E6444FF651
:10126000FF7C0CEA05252C430D8922F020020CEAB4
:1012700005152A434D880CEA05152A43A0F180453F
:10128000B5F596351CBFA0F18045B5F59A3516D158
:101290004D8922F080020CEA05152A438D8822F040
:1012A00040020CEA05152A438D8923F440630CEAB9
:1012B00085052B43CD890CEA850C4CEA030383801A
:1012C0000483C9880187028430BC704730B4028C23
:1012D00022F480520284038C8288B0F81CC00D88EE
:1012E0004FF6FF742CF4E64C04EA052545EA0C0C95
:1012F0000D8923F4005304EA05352B434D8804EA95
:1013000005352B43A0F18045B5F596351CBFA0F1FE
:101310008045B5F59A3505D18D8922F4804204EADD
:10132000851422438280A0F81CC0C988A0F8401010
:10133000038430BC7047828B4FF6FF7322F4006247
:1013400003EA012111438183704781857047A0F82A
:101350004010704710B40288DFF88CC0234B604502
:1013600018BF984211D0B0F1804F1CBFA0F180444B
:10137000B4F5806409D0A0F18044B4F500641CBFCA
:10138000A0F18044B4F5406403D14C8822F070028F
:101390002243A0F18044B4F580541CBFA0F18044E6
:1013A000B4F5A05403D0CC8822F4407222430280CA
:1013B0008A8882850A880285604518BF98420DD0C8
:1013C000A0F18042B2F5A0321FBFA0F18042B2F579
:1013D000A232A0F18042B2F5A43201D1097A01868D
:1013E0000121818210BC7047002C01400034014073
:1013F0004FF6FF71818000210180C1804180017220
:101400007047C9B28180018811F0800FFBD070470E
:10141000FEE72DE9F05F0A46C16900278B1CC0E991
:1014200006130A80858A0269C36902EB45013E46BC
:10143000994208BFC2610023D0F820C004686FF051
:101440000109816934F913A0A1F10208C0F81880DC
:10145000B1F90010904504D209EB45089044C0F85A
:1014600018800AFB01F1CF1946EBE17803F1010185
:1014700034F911A08169A1F102068661B1F9001069
:10148000964203D209EB4506164486610AFB01F138
:10149000CF1948EBE17803F1020134F911A0816919
:1014A000A1F102068661B1F90010964203D209EB60
:1014B0004506164486610AFB01F1CF1948EBE17835
:1014C00003F1030134F911A08169A1F102068661DB
:1014D000B1F90010964203D209EB45061644866125
:1014E0000AFB01F1CF1948EBE17603F10403BCF1EB
:1014F000010CA6D1D0F824A0BAF1000F1AD90CEB38
:10150000030134F911B08169A1F10208C0F8188013
:10151000B1F90010904504D209EB45089044C0F899
:1015200018800BFB01F1CF1946EBE1760CF1010CB1
:10153000E245E4D8B0F928203846D3173146FEF703
:1015400048FE00B2BDE8F09F2DE9F0470546026075
:1015500081800020A8712868A860E860481C87B2D4
:10156000780098460E4605F11004814600F074FAA2
:101570002060A7800120A0712068A0604946E0603B
:10158000FEF74BFEB008286206F003006862A5F87B
:1015900028802846BDE8F0870446032100F016FAAB
:1015A000012104F1340000F06FF904F1340000F07F
:1015B0002DFA01B2201DFFF72CFF00F5006081B26B
:1015C00004F1300000F032FAEFE7000010B500F04F
:1015D00015F943F6FF730A4A1F21001DFFF7B4FFF8
:1015E00001212C3000F0BCF90321001D00F050F95E
:1015F000A0F13404642100F021F9204610BD000060
:101600004C1B000810B50446124A00200029107037
:1016100004BF30BF10BD02210120FFF7E7FA4FF4ED
:101620008030FFF757FBFFF781FB2060012818BFD0
:1016300010BD0120FFF76AFB3920FFF72BFB0028C4
:10164000FAD00220FFF768FBFFF73CFB0828FBD12C
:1016500010BD00000000002030B58BB00121022039
:10166000FFF7E8FA4FF40070ADF81C00182009905D
:101670000220089007A91D48FFF7DEF901211C4848
:10168000FFF73AFA1B4D2846FFF797FC42F6E06158
:101690004FF47A70ADF81410ADF810000024ADF8D6
:1016A0001640ADF8124004A92846FFF753FE60210A
:1016B000ADF800100121ADF8021041F27071ADF8E3
:1016C0000610ADF8084069462846FFF7FFFD0821DF
:1016D0002846FFF730FE01212846FFF759FC01217B
:1016E0002846FFF761FC0BB030BD00000010014040
:1016F000000C1A000004004070B58AB001210420DB
:10170000FFF798FA194E3046FFF757FC4FF6FF7077
:10171000ADF8040045F6C050ADF800000024ADF867
:101720000640ADF8024069463046FFF713FE102030
:10173000ADF810000125ADF81250ADF8184004A91D
:101740003046FFF73EFD1E208DF820008DF8224028
:1017500004208DF8210008A80995FFF70BFA012253
:1017600002213046FFF725FD0AB070BD0008004099
:1017700070B4184D2B68012000FA02F223EA02002F
:10178000154BD3F800C04CF0807CC3F800C0DFF8E4
:1017900050C0124BCCF800302860124C4FF0000CB7
:1017A000C4F800C0104B0226C3F8F060491E19614E
:1017B0000E49C1F800C0DFF83CC00D49CCF800105C
:1017C0008915C3F804130C4921601043286070BCCC
:1017D00070470000000E00E0FCED00E055CEACC507
:1017E000B00F00E0800E00E0000004E0400E00E0DA
:1017F000FE030040001000E00D00010010B504469B
:1018000072B600220821FFF7B3FF0020FFF7AAFA03
:101810000020FFF7C7FA0120FFF7A4FA0120FFF725
:10182000C1FA01210020FFF7D5FA2046FFF764FF37
:101830002046FFF711FF62B6204610BD30B589B0D3
:1018400005460C466846FFF7D3FD1820ADF80000AA
:101850000020ADF80440ADF80600ADF8020069467E
:101860002868FFF777FD6020ADF810000120ADF883
:1018700012000220ADF81640ADF8180004A928683F
:10188000FFF7E1FC09B030BD0068FFF78DBB000039
:10189000F0B5044689B04FF08040206001200E462C
:1018A00060604FF4C020C4E9020601214802FFF73E
:1018B000D9F9284DD5E906012A6ACDE90601281D86
:1018C000089230F81600ADF8180006A92248FFF774
:1018D000B3F82846865D0020FFF7A2F91F4F38466F
:1018E000FEF72BFF05F124000FC88DE80F00D5E9A6
:1018F0000D01CDE90401A068039069463846FEF762
:101900006DFF0723012231463846FEF78BFF012188
:101910003846FEF740FF01216068FFF78BF9002190
:101920002068FFF741FB01213846FEF7FDFE3846EF
:10193000FEF7C0FF3846FEF749FF0028FAD13846C7
:10194000FEF7BDFF3846FEF72FFF0028FAD109B099
:101950002046F0BDF41A00080008014000240140B0
:1019600030B587B00C460160054601214807FFF7F6
:1019700061F9FEF7B9FF1348012CD0E90312406961
:101980000491CDE905200CBF20201020ADF81000F7
:1019900004A90D48FFF750F8002000900190029034
:1019A0000390012C0CBF102000206946FEF7A8FF11
:1019B000012C0CBF102000200121FEF787FF07B08B
:1019C000284630BDF41A00080008014070B50D48E3
:1019D00099B10D4A054632F811400121FFF7E4FAAA
:1019E0004FF6FF7101EA44012846FFF7AEFC21469D
:1019F0002846BDE87040FFF7AABCBDE87040002152
:101A0000FFF7D2BA00040040E81A000810B5064CEF
:101A100002212046FEF7D3FE0028F9D02046BDE87B
:101A20001040FEF7C9BE000000240140B1F5805F00
:101A300028BF40F6FF71006801284FF0000001D078
:101A4000FEF778BFFEF781BF10B500F001F810BDBA
:101A500010B5FEF7D8FC10BD10B500F001F810BDB0
:101A600010B5040007D1012405E0FEF799FC0068D9
:101A700000B9044880472046FEF796FC0028F4D0C1
:101A800010BD000055040008FEE700F023B800B5C3
:101A900091B000216846FFF799FD00216846FFF7E5
:101AA00095FF00216846FFF7ADFD6846FFF774FD1E
:101AB0009DF81A00012804BF0598FFF7C5FF9DF89F
:101AC0000A00012804BF0198FFF7BEFF002011B0F3
:101AD00000BD000010B5044681B20248FFF791FC3A
:101AE000204610BD003801400000E02E7017B80BF2
:101AF000E8030000010203060200040008004000A1
:101B000000000000020000001000000000000000C3
:101B100003000000000000000000000000000000C2
:101B200000000000000000000000000001000000B4
:101B3000000000000100010006000002000100009A
:101B4000040000001000000010000000E5FF1F006E
:101B50004C00D6FF2AFF0000C101BC0049FDCDFDAD
:101B600023031B0473FD41FAFC006606FC0041FAE6
:101B700073FD1B042303CDFD49FDBC00C101000022
:101B80002AFFD6FF4C001F00E5FF0000AC1B000839
:101B9000000000201000000028010008BC1B000805
:101BA0001000002060060000440100080000000052
:0C1BB0000008014000100140001001403E
:04000005080000ED02
:00000001FF
